:1000000042C0ADC15BC05AC059C058C057C056C0ED
:1000100055C054C053C052C051C050C04FC04EC054
:100020004DC04CC04BC04AC049C048C047C046C084
:1000300045C044C0040309041C037700770077001F
:100040002E00660069007300630068006C002E00DB
:10005000640065000E035500530042006100730008
:10006000700012011001FF000008C016DC05040139
:1000700001020001090212000101008019090400B7
:1000800000000000000011241FBECFEFD4E0DEBF4F
:10009000CDBF11E0A0E0B1E0E8E7F2E102C00590D9
:1000A0000D92A230B107D9F711E0A2E0B1E001C092
:1000B0001D92AA34B107E1F767D5DCC8A1CFE9E604
:1000C000F0E0808182608083E89A08951F93CF9347
:1000D000DF9360912801635067FD13C08091250173
:1000E000CCE0D0E0C81BD109C45DDE4F8091240173
:1000F0008D3209F462C08091020187FD84C01092A4
:1001000028018091000184FF4AC0609101016F3F86
:1001100009F445C0693070F1685060930101809125
:10012000180198E889278093180168E080910201FE
:1001300087FD8BC0209126013091270186FF6DC07D
:10014000A9E1B1E080E090E0F901E80FF91FE49146
:10015000ED9301966817C1F76150862F90E06F5FAD
:100160000196820F931F9093270180932601162FEB
:100170001C5F0BC0109201018091180198E889273B
:1001800080931801662391F614E089E191E0E3D0B1
:100190001C3019F08FEF809301011093000194E15E
:1001A00089B1847131F49150D9F7109229011092DC
:1001B0002301DF91CF911F910895683009F09FCFFF
:1001C00083EC809318018AE580930001109202016C
:1001D0008881807659F59A8110922101898188233E
:1001E00009F043C01092220122E081E291E0909355
:1001F0002701809326018F81882319F49E8192170D
:1002000008F1922F1FC0CE01D7D48F3F51F1882320
:1002100009F475CF1092010172CFD901962FE9E14F
:10022000F1E08D9181939150E1F796CFCE010CD6FC
:10023000282F8F3F01F7888187FD25C09FEF80E839
:1002400080930201909301015ACF89E191E08AD510
:10025000682F893008F453C08FEF809301011EE1AD
:100260009CCF8EE1809300014ACF853071F08630BB
:1002700091F0883031F1893061F18A3031F120E03C
:1002800081E291E0B4CF9E81DACF9093290120E002
:1002900081E291E0ACCF8B81813049F18230F9F07D
:1002A000833029F020E080E480930201A4CF9923D9
:1002B00049F584E390E0909327018093260124E0A0
:1002C000F2CF21E08BE291E092CF21E081E291E058
:1002D0008ECF90932B0120E081E291E088CF84E7DC
:1002E00090E0909327018093260122E1DCCF82E603
:1002F00090E0909327018093260122E1D4CF182F1C
:100300001C5F43CF913051F0923061F684E590E06C
:1003100090932701809326012EE0C5CF88E390E0DB
:1003200090932701809326012CE1BDCFA82FB92FF0
:1003300080E090E041E050EA609530E009C02D9106
:1003400082279795879510F084279527305EC8F30C
:100350006F5FA8F30895EADF8D939D930895CF937F
:10036000CFB7CF93C3954C9BE9F74C9B09C04C9BEF
:1003700007C04C9B05C04C9B03C04C9B01C0A1C057
:10038000DF93C0912501DD27C45DDE4F4C9B02C089
:10039000DF91EBCF2F930F931F9309B12FEF04FB46
:1003A00020F94F933F9319B14FEF012704FB21F937
:1003B0003BE031C04E7F012F19B1216028C0102FC2
:1003C0004D7F2260000009B129C04B7F2460012FBE
:1003D000000019B12BC019B1477F28602AC04F7E99
:1003E00009B120612CC04F7D19B120622FC04F7B15
:1003F00009B1206432C0422709B149934FEF000090
:10040000102714FB20F919B11471C9F1297F91F259
:10041000012704FB21F909B1237F89F2315058F1FA
:10042000102714FB22F919B1277E79F2012704FB6A
:1004300023F92F7C81F209B1102714FB24F92F79BD
:1004400071F200C019B1012704FB25F92F7359F28D
:1004500000C009B1102714FB26F9223040F200C079
:1004600019B1012704FB27F9243028F64F772068BB
:1004700019B10000F9CF11E01CBB002717C03B5099
:100480003195C31BD04011E01CBB0881033CE9F04F
:100490000B34D9F0209123011981110F1213EDCFE4
:1004A000093641F10D3211F0013E39F700932A016E
:1004B0003F914F911F910F912F91DF91CCB3C0FDD0
:1004C00051CFCF91CFBFCF91189520912A012223F0
:1004D00079F310912801112311F5343012F1309382
:1004E000280120932401109125013BE0311B30931A
:1004F000250117C00091280101308CF40AE53091E4
:10050000000134FD10C000930001C8E1D1E00FC02C
:100510002795A8F45150A9F4220F0000F9CF4AE51D
:1005200003C042ED01C0432FC4E1D0E032E01AB174
:1005300014615C9A1AB90BB120E414E15F930127AE
:1005400056E00BB9279520F4515021F4220FF9CF32
:10055000012756E000003B5A0BB9D0F2279528F44A
:10056000515029F4220F0000F9CF012756E02795BA
:100570000BB920F4515021F4220FF9CF012756E096
:10058000299133230BB921F60B7E10912901110F0C
:10059000C651D0400BB911F01093230111E01CBBE0
:1005A00000611AB11B7E402F4B7E5F9100C000C0DE
:1005B0000BB91AB94BB97CCF809145018CBD8091A4
:1005C00042018DBD0895282F8823A1F0883008F0BE
:1005D00042C085E893E09093440180934301243026
:1005E00019F12530B8F0263099F1263068F127301E
:1005F000F9F0089586EA93E09093440180934301D3
:1006000081E08093470182E58093450181E08093FA
:10061000420108952230A1F0233070F4213049F7CF
:1006200080EC80934701089588E180934701089505
:1006300083E080934701089580E380934701089504
:1006400080E68093470108958CE0809347010895E8
:1006500020934701089586EA93E0909344018093A4
:1006600043011092420181E080934701293041F01B
:100670002A3050F4283039F683E5809345010895F7
:1006800082E58093450108952B3029F02C3009F044
:10069000BACF8093420181E580934501089526B544
:1006A0009091470186B5821B8917E0F3089584B1C4
:1006B0008C6284B92A982D9896B52091470186B509
:1006C000891B8217E0F32A9A96B586B5891B821793
:1006D000E0F32A988091430190914401865A934017
:1006E00019F0109246010895809145018CBD8091CA
:1006F00042018DBD10924601089584B1837D84B975
:1007000085B1837D85B91CBC0895582F2091470180
:1007100040E030E057FD16C02B98440F1C994F5F06
:100720002D9A96B586B5891B8217E0F32D9896B55C
:1007300086B5891B8217E0F33F5F383029F0550FEB
:1007400057FFEACF2B9AE9CF842F08958EBD0DB4C1
:1007500007FEFDCF8EB508950F931F930FE1E09133
:100760004301F09144018CEA0995E0914301F09135
:10077000440183E50995E0914301F091440180E053
:100780000995182FE0914301F091440180E009950B
:10079000133561F11CBC26B59091470186B5821BCB
:1007A0008917E0F32A9A26B586B5821B8917E0F3EC
:1007B0002A9826B586B5821B8917E0F3E09143019C
:1007C000F091440183E0E63AF80721F0002351F06C
:1007D0000150C9CF809145018CBD809142018DBDF2
:1007E0000023B1F781E01F910F91089580E01F91E0
:1007F0000F9108959B01AC0181E15695479537957E
:1008000027958A95D1F7809146018217D9F02093D8
:100810004601E0914301F09144018DE40995E09196
:100820004301F091440180E00995E0914301F0918A
:100830004401809146010995E0914301F091440102
:1008400080E009950895EF92FF920F931F937B012B
:100850008C01D0DF8E2D8170880F880F880FE0917A
:100860004301F091440180620995D801C70129E054
:10087000B695A795979587952A95D1F7E09143016D
:10088000F0914401099516950795F794E794E09146
:100890004301F09144018E2D0995E0914301F091BF
:1008A000440180E009951F910F91FF90EF9008950A
:1008B0000F931F938C01E0914301F091440180EA72
:1008C0000995E0914301F0914401812F0995E09150
:1008D0004301F0914401802F0995E0914301F0918B
:1008E000440180E009951F910F910895FF920F93A5
:1008F0001F938C01F62EE0914301F091440180ECAE
:100900000995E0914301F0914401812F0995E0910F
:100910004301F0914401802F0995E0914301F0914A
:1009200044018F2D09958EE1B9D080E01F910F9180
:10093000FF900895CF92DF92EF92FF920F931F9353
:100940006B017C01142F56DFE0914301F0914401CB
:100950008CE40995D701C60149E0B695A79597950E
:1009600087954A95D1F7E0914301F09144010995AB
:10097000D701C601B695A79597958795E091430154
:10098000F09144010995E0914301F091440180E028
:1009900009951F3FF1F016B50EE1C701B60153DF0F
:1009A0008F3F79F486B5811B8D33B8F316B50150AE
:1009B000A1F781E01F910F91FF90EF90DF90CF9012
:1009C000089580E01F910F91FF90EF90DF90CF90FE
:1009D00008958FE063D080E01F910F91FF90EF901A
:1009E000DF90CF900895CF92DF92EF92FF920F9316
:1009F0001F936B017C01042F122FFCDE8C2D817064
:100A0000880F880F880FE0914301F09144018064C2
:100A10000995D701C60169E0B695A7959795879581
:100A20006A95D1F7E0914301F09144010995D7010E
:100A3000C601B695A79597958795E0914301F091EA
:100A400044010995E0914301F0914401802F0995FB
:100A50001123C1F00F37F1F016B50EE1C701B60151
:100A6000F2DE8F3779F486B5811B8D33B8F316B576
:100A70000150A1F781E01F910F91FF90EF90DF905F
:100A8000CF90089580E01F910F91FF90EF90DF903D
:100A9000CF9008958FE002D080E0F5CF382F8823E3
:100AA00049F020E096B586B5891B8C33E0F32F5FC3
:100AB0002317C0F30895259A23982B9A50E217D054
:100AC0005A95E9F70895AC0188E605D0842F03D044
:100AD00089E601D0852F0FD028E030E0382780FB51
:100AE000869506D02A95D1F730FB02D000D06894C5
:100AF00023982B9A16F02B98239AE0914801F091B5
:100B000049013197F0F72D9AE3B1E3FBE0914801F9
:100B1000F09149013197F0F72D98089520ECE7DF27
:100B200046F42A95E1F780E02AE1E5DF2A95E9F726
:100B3000DECF28E030E0DBDF869587F938272A957D
:100B4000D1F7D5DF27F9322772F3D1DFD0CFDB0120
:100B5000742FB9DF84E2BFDFE1DF8D937A95D1F79F
:100B60000895DB01742FAFDF83EFB5DF8DE1B3DFD5
:100B700084E6B1DF8D91AFDF82E7ADDFCFDF807834
:100B8000D9F77A9589F7089593E095B98CE388B9F8
:100B90008AEE8BB9389A399A4198409A5098589A67
:100BA0008AB184618AB98AB18B7E8AB995BD87DAA8
:100BB00078948CDA8BDAFDCFFF920F931F93CF934B
:100BC000DF93082F792FF62E40910301413069F011
:100BD000443059F0463009F492C01FEF812FDF9165
:100BE000CF911F910F91FF900895FF2009F4B2C09B
:100BF000802F972F9C01E90110E053C080911401D0
:100C000090911501892B09F058C0609110017091E5
:100C100011018091120190911301488121E0E3DEDE
:100C200080910401909105010197909305018093B3
:100C30000401892BD9F4109203018091160181FFE0
:100C40003AC08091170190E0209114013091150174
:100C50008217930781F160911001709111018091C9
:100C6000120190911301488165DE11E0809110011D
:100C700090911101A0911201B09113010196A11D53
:100C8000B11D8093100190931101A0931201B093B4
:100C9000130121969E01201B2F1508F09FCF409134
:100CA0000301413009F4AACF809110019091110104
:100CB00068811CDEB5CF11E0D9CF60911001709131
:100CC00011018091120190911301488120E08BDE87
:100CD00080911701815080931701882309F0A0CFDC
:100CE0006091100170911101809112019091130196
:100CF000488120DE809114018093170191CF80916B
:100D0000100190911101602F4F2D2BDF8091100168
:100D100090911101A0911201B09113018F0D911DBD
:100D2000A11DB11D8093100190931101A093120198
:100D3000B093130180910401909105018F199109DD
:100D40009093050180930401892B21F410920301F3
:100D500011E044CF10E0812FDF91CF911F910F91CF
:100D6000FF9008950F931F93CF93DF93082F792F50
:100D7000162F40910301842F8250823050F045306D
:100D800009F446C01FEF812FDF91CF911F910F9182
:100D900008954530E9F1662399F1802F9C01E9011E
:100DA00020C0809110019091110182DD8883809193
:100DB000100190911101A0911201B09113010196BF
:100DC000A11DB11D8093100190931101A0931201F8
:100DD000B093130121969E01201B211778F44091B6
:100DE00003014230F1F66091100170911101809180
:100DF00012019091130127DD8883D9CF183018F69E
:100E000010920301812FDF91CF911F910F910895CF
:100E10008091100190911101602F412F98DE8091F7
:100E2000100190911101A0911201B0911301810F55
:100E3000911DA11DB11D8093100190931101A093EC
:100E40001201B09313019FCF0F931F93CF93DF93A2
:100E50008C01DC0111968C91813009F44EC08230F6
:100E600009F4E7C0833009F455C0843009F4B5C0F3
:100E7000873009F486C0853009F45AC1863009F4F8
:100E800010C1883009F4DBC0893009F458C18A30B8
:100E900009F469C18B3009F49CC18C3009F4B7C1E5
:100EA0008D3009F4CBC18E3009F4CFC18F3009F0F9
:100EB00065C1F801938180E0228130E0822B932B81
:100EC000AA2797FDA095BA2F809310019093110146
:100ED000A0931201B0931301978180E0268130E046
:100EE000822B932B909305018093040185E08093DE
:100EF00003018FEFC8E0D1E038C0489B3FC080912C
:100F0000060161DB109207014098D1DB80E0C8E068
:100F1000D1E02BC0E0914301F0914401D801129639
:100F20008C910995C8E0D1E080930801E0914301DC
:100F3000F0914401D80113968C9109958093090191
:100F4000E0914301F0914401D80114968C910995E8
:100F500080930A01E0914301F0914401D801159674
:100F60008C91099580930B0184E0D0932701C09365
:100F70002601DF91CF911F910F91089585E023DB2A
:100F8000C1CF80910701882399F4F801938180E013
:100F9000228130E0822B932BAA2797FDA095BA2FB0
:100FA0008093100190931101A0931201B09313014B
:100FB000D80117969C91179780E016962C9130E0F7
:100FC000822B932B909305018093040183E08093FF
:100FD00003018FEFC8E0D1E0C8CF809107018823DB
:100FE00099F4F801938180E0228130E0822B932BE9
:100FF000AA2797FDA095BA2F809310019093110115
:10100000A0931201B0931301D80117969C911797E2
:1010100080E016962C9130E0822B932B9093050163
:101020008093040182E0809303018FEFC8E0D1E058
:101030009CCF63DB409A80E0C8E0D1E096CF8091FE
:1010400007018823B1F4D80113969C91139780E08F
:1010500012962C9130E0822B932BAA2797FDA09516
:10106000BA2F8093100190931101A0931201B093B5
:101070001301109215011092140110921601F8013B
:10108000978180E0268130E0822B932B909305019D
:101090008093040184E0809303018FEFC8E0D1E0E6
:1010A00064CF80910701882399F4F801938180E04F
:1010B000228130E0822B932BAA2797FDA095BA2F8F
:1010C0008093100190931101A0931201B09313012A
:1010D000D80114968C91149715969C91292F2F70F6
:1010E00020931601492F50E0407F50704295529551
:1010F000507F5427407F5427480F511D50931501AE
:101100004093140120FF02C040931701F80197811A
:1011100080E0268130E0822B932B90930501809311
:10112000040181E0809303018FEFC8E0D1E01DCF7F
:1011300013DBC8E0D1E08093080181E016CF81E0A5
:1011400080930701F80182819381A481B581809306
:10115000100190931101A0931201B093130180E04C
:10116000C8E0D1E002CFD80112968C91809306019D
:10117000C8E0D1E01092080181E0F7CE803109F09B
:1011800040C0D80113969C91139780E012962C9141
:1011900030E0822B932BAA2797FDA095BA2F80933E
:1011A000100190931101A0931201B0931301F80163
:1011B000978180E0268130E0822B932B909305016C
:1011C0008093040186E0809303018FEFC8E0D1E0B3
:1011D000CCCEF801938180E0228130E0822B932BEA
:1011E00090934901809348012A9A229A83E056DC21
:1011F0002A98409880E152DC5EDC80E0C8E0D1E0D3
:10120000B4CE8F3751F180E0C8E0D1E0AECE80ECB3
:1012100062DC80E060DC8AE041DC2A9A85E03EDC2A
:101220002A9885E03BDC84B1837D84B985B1837DD8
:1012300085B9409A80E0C8E0D1E097CE6FDCC8E085
:10124000D1E08093080181E090CED80112968C9174
:1012500042DC80E0C8E0D1E088CEC8E0D1E081E0A7
:10126000809308011092090110920A0110920B015B
:0812700084E07BCEF894FFCF6F
:021278005AFF1B
:00000001FF
